:1000000051282D3094000C3095003C309600960B12
:100010000728950B0528940B032896309400940B21
:100020000F28000000000800113094000D309500EA
:100030003A309600960B1A28950B1828940B162820
:10004000C5309400940B22280000000008004230C4
:100050009400940B292808000A309400423095003F
:10006000950B3028940B2E280800851005103A288F
:10007000851005149A000310083093009A0D900C17
:10008000930B3E2810088600851400008510272059
:100090002720100E860085140000851027202720B9
:1000A000080083018316B73081001C308500F030D2
:1000B0008600831285018601012005108510043019
:1000C000860085140000851027200C3035202C2058
:1000D000283035202C20013035202C20C030352010
:1000E0002C20920112088900831608148312080834
:1000F0003820920A121E72288C3035202C204D3068
:100100003820683038207A303820860186149701EC
:10011000FF30980099008101861006158615012090
:100120000120012001200120012014200611861148
:1001300001089700910083018316861383128617A6
:1001400000008613000011080106031DA92898036A
:100150009F2883018316861783120000861BB92807
:100160000615000006110000861BB8289903B02868
:1001700099030615000006110000861FC128990387
:10018000B9289903183093008C018D018E018F01DD
:100190000310990D980D970D8C0D8D0D8E0D8F0DF3
:1001A000930BD328EB280F308400E0200E3084001E
:1001B000E0200D308400E0200C308400E020C928CD
:1001C0000330000791009119800030300007910042
:1001D000911B80000800823035202C2030309100A7
:1001E0000F0E0F39031DFC28203038200F080F395F
:1001F000031D002920300129110738200F080F396D
:10020000110738200E0E0F39110738200E080F394C
:10021000110738202E3038200D0E0F3911073820E5
:100220000D080F39110738200C0E0F39110738202F
:0A0230000C080F391107382085284B
:02400E00F93F78
:1042000020004600310047004C00540020002000F0
:1042100020004A004E0031003600520056002000B7
:00000001FF
